:020000040800F2
:100000009805002089020008910200089302000868
:1000100095020008970200089902000800000000FD
:100020000000000000000000000000009B0200082B
:100030009D020008000000009F02000891130008C4
:10004000A3020008A3020008A3020008A3020008FC
:10005000A3020008A3020008A3020008A3020008EC
:10006000A3020008A3020008A3020008A3020008DC
:10007000A3020008A3020008A3020008A3020008CC
:10008000A3020008A3020008A3020008A3020008BC
:10009000A3020008A3020008A3020008A3020008AC
:1000A000A3020008A3020008A3020008A30200089C
:1000B000A302000861140008A3020008A3020008BC
:1000C000A3020008A3020008A3020008A30200087C
:1000D000A3020008B5170008A3020008A302000845
:1000E000A3020008A3020008A3020008A30200085C
:1000F000A3020008A3020008A3020008A30200084C
:10010000A3020008A3020008A3020008A30200083B
:10011000A302000881160008A3020008A302000839
:10012000A3020008A3020008A3020008A30200081B
:10013000A3020008A3020008A3020008A30200080B
:10014000A3020008A3020008A3020008A3020008FB
:10015000A3020008A3020008A3020008A3020008EB
:10016000A3020008A3020008A3020008A3020008DB
:10017000A3020008A3020008A3020008A3020008CB
:10018000A3020008A302000800F002F800F064F8DF
:100190000AA090E8000C82448344AAF10107DA45E2
:1001A00001D100F059F8AFF2090EBAE80F0013F0D0
:1001B000010F18BFFB1A43F001031847481C000049
:1001C000681C00000A444FF0000C10F8013B13F0CB
:1001D000070408BF10F8014B1D1108BF10F8015BA0
:1001E000641E05D010F8016B641E01F8016BF9D193
:1001F00013F0080F1EBF10F8014BAD1C0C1B09D1EA
:100200006D1E58BF01F801CBFAD505E014F8016B5B
:1002100001F8016B6D1EF9D59142D6D370470000ED
:100220000023002400250026103A28BF78C1FBD8FF
:10023000520728BF30C148BF0B607047642900F0E7
:100240008380782900F0BC80002070471FB501F042
:10025000BFFC1FBD10B510BD00F0FEF91146FFF741
:10026000F5FF01F0BDFB00F01CFA03B4FFF7F2FF4D
:1002700003BC01F0A5FB000030BF72B6704762B648
:10028000704780F30888704709488047094800474D
:10029000FEE7FEE7FEE7FEE7FEE7FEE7FEE7FEE736
:1002A000FEE7FEE704480549034A054B7047000096
:1002B000A11300088901000898010020980500207A
:1002C00098010020704700000FB4044910B503AA3C
:1002D000029800F06BF910BC5DF814FB00000020E0
:1002E0002DE9F0410E460446002020622046E168D8
:1002F000884730B3252805D0D4E901219047206AEA
:10030000401CF2E7E168204600278847050018D026
:10031000A5F14100192802D820354FF40067324674
:10032000294620462760FFF789FF40B1012804D005
:10033000F61D26F007060836D8E7361DD6E728460C
:10034000DAE7206ABDE8F0812DE9F0410646002495
:1003500010687529314616A510D0AFF3008000282B
:1003600002DA404213A507E031688A0701D512A5D9
:1003700002E0490704D511A5012401E0AFF3008094
:1003800000210A2206F1240709E0B0FBF2FCB0FBD1
:10039000F2F302FB1C00303078541846491C002848
:1003A000F3D123462A463046BDE8F04100F0A5B817
:1003B000000000002D0000002B00000020000000C5
:1003C00070B504460D4621461068AFF300802188C1
:1003D000090502D50F4A7A4402E00E4A7A440E32E9
:1003E000002104F1240305E000F00F060009965DEA
:1003F0005E54491C0028F7D120780023000704D55B
:10040000702D02D009B1022311322046BDE87040A0
:1004100000F073B8001A000040EA010370B59B07B2
:100420002ED14FF00136042A2AD308C810C99D1BCB
:100430009D43121F15EAC61517D0D8B2E1B2401A73
:1004400050EA056110D198B2A1B2401A50EA0541B4
:100450000AD123F07F4024F07F41401A50EA052161
:1004600002D1180EA0EB146070BDA342DBD018BA05
:1004700021BA884201D9012070BD4FF0FF3070BD14
:100480000AB9002070BD10F8013B11F8014B63B1AF
:10049000A3420AD1521E08D010F8013B11F8014BBB
:1004A0001BB1A34201D1521EEDD1181B70BD4FF0FC
:1004B00000020429C0F0128010F0030C00F08A80C2
:1004C000CCF1040CBCF1020F18BF00F8012BA8BF3F
:1004D00020F8022BA1EB0C0100F07CB85FEAC17C94
:1004E00024BF00F8012B00F8012B48BF00F8012BB6
:1004F000704770477047704770472DE9F0470D46C9
:1005000099469246044600F124080168880604D5FD
:10051000E06921F01001216000E00120A84201DD26
:10052000471B00E00027A1697A1902EB0900081AAD
:10053000A0612078C00602D42046AFF300800026D8
:1005400008E0D4E901211AF806009047206A401C0F
:10055000761C20624E45F4DB2078C0060AD5204682
:10056000AFF3008006E0D4E9012130209047206AF3
:10057000401C2062381EA7F10107F4DC07E0D4E933
:10058000012118F805009047206A401C2062281EAF
:10059000A5F10105F3DC2046AFF3008020780006CA
:1005A00002D50220BDE8F0870120FBE7074B70B5BC
:1005B0000D467B4400F039F80446284600F048F820
:1005C00010B14FF0FF3070BD204670BD0F14000019
:1005D0004FF0000200B5134694469646203922BFDC
:1005E000A0E80C50A0E80C50B1F12001BFF4F7AF27
:1005F000090728BFA0E80C5048BF0CC05DF804EB09
:10060000890028BF40F8042B08BF704748BF20F876
:10061000022B11F0804F18BF00F8012B704700002B
:1006200001694A1C02610878704700B58FB0CDE9B6
:1006300001310021059105497944CDE903101146A6
:100640006846FFF74DFE0FB000BD0000E5FFFFFF5D
:10065000007B00F080007047754600F02BF8AE4636
:1006600005006946534620F00700854618B020B5BE
:10067000FFF718FEBDE820404FF000064FF00007DE
:100680004FF000084FF0000B21F00701AC46ACE83A
:10069000C009ACE8C009ACE8C009ACE8C0098D46A7
:1006A000704710B50446AFF300802046BDE8104007
:1006B000FFF7DBBD004870473401002010B5044847
:1006C00001680448FFF7F3FE00200149086010BDEF
:1006D00004000020000000687FB5684600F008FDB7
:1006E0004FF47A720098B0FBF2F1481EB0F1807FAF
:1006F00000D31BE0481E4FF0E022506150170F223C
:10070000002807DA13071D0E094B00F00F04241F01
:100710001D5503E013071C0E064B1C5400BF0020A0
:100720004FF0E02290610720106100BF7FBD000004
:1007300018ED00E000E400E010B5002418E04FF4EC
:100740007A7000F011FF0C48007878B100200A4957
:100750000870072209A10B48FFF75EFE30B915218A
:10076000094801F009F900F051FB03E0601CC4B234
:10077000052CE4DB00BF10BD0C00002055504441A7
:1007800054450000000000681F01002030B10749F7
:10079000096841F48061054A116005E00349096870
:1007A00021F48061014A116070470000003C024062
:1007B00070B504460A460026092502B909E0012A57
:1007C00001D1160205E0022A01D1160201E04FF420
:1007D000407600F09FF80546092D28D1154800689D
:1007E00020F44070134908600846006830430860F0
:1007F0000846006820F0F80008600846006844F0E9
:10080000020108430B4908600846006840F4803044
:10081000086000F07FF805460648006820F00200F6
:10082000044908600846006820F0F800086028467F
:1008300070BD0000103C024009201349096801F412
:100840008031B1F5803F01D101201CE00E490968DB
:1008500001F0100109B1062015E00B49096801F407
:10086000807109B102200EE00749096801F0EF012B
:1008700009B1072007E00449096801F0020109B144
:10088000082000E0092070470C3C02400348006843
:1008900040F000400149086070470000103C0240F1
:1008A00030B502460C46092500F034F80546092DFE
:1008B00019D10E48006820F440700C4908600846C1
:1008C000006840F4007008600846006840F00100CD
:1008D0000860146000F01EF805460448006820F027
:1008E000010002490860284630BD0000103C02406B
:1008F0000548006800F0004028B1044802490C395E
:100900000860034808607047103C024023016745B7
:10091000AB89EFCD08B509200090FFF78DFF00905F
:1009200002E0FFF789FF00909DF800000128F8D051
:100930009DF8000008BD000051B18200A2F1C04244
:10094000126842F001038200A2F1C042136009E084
:100950008200A2F1C0421268034B1A408300A3F147
:10096000C0431A6070470000FEFF0F00D0E901127B
:100970001143C268114302691143426911438269FC
:100980001143C2691143026A1143426A1143826AE8
:100990001143C26A1143026B114302689200A2F133
:1009A000C0421160816808290BD101688900A1F15A
:1009B000C041096841F0400201688900A1F1C041CD
:1009C0000A60416B0968426B526841EA0211426B4E
:1009D000926841EA0221426B928941EA0241426BEC
:1009E000128A41EA0251426B127D41EA0261426B76
:1009F000926911430268521C9200A2F1C042116038
:100A0000C16AB1F5804F1BD1816B0968826B526856
:100A100041EA0211826B926841EA0221826B128ADA
:100A200041EA0251826B127D41EA0261826B926956
:100A3000114302689200A2F1C042C2F8041107E01B
:100A40006FF0704201688900A1F1C041C1F8042132
:100A50007047000000B599B001217A2000F008FB32
:100A60000121084600F014FB4FF6B37017900220E6
:100A70008DF8600000208DF8620003208DF8610081
:100A800001208DF8630017A9964800F033F94FF65E
:100A90008370179002208DF8600000208DF86200AE
:100AA00003208DF8610001208DF8630017A98E489E
:100AB00000F020F94FF23F00179002208DF86000FF
:100AC00000208DF8620003208DF8610001208DF870
:100AD000630017A9854800F00DF93F201790022008
:100AE0008DF8600000208DF8620003208DF8610011
:100AF00001208DF8630017A97D4800F0FBF80C2257
:100B00000021784800F03EF90C220121754800F0E0
:100B100039F90C220421734800F034F90C22052124
:100B2000704800F02FF90C2208216E4800F02AF9D5
:100B30000C2209216B4800F025F90C220A21694892
:100B400000F020F90C220B21664800F01BF90C2262
:100B50001146644800F016F90C220D21614800F09E
:100B600011F90C220E215F4800F00CF90C220F2124
:100B70005C4800F007F90C2200215B4800F002F904
:100B80000C220121584800F0FDF80C22072156489C
:100B900000F0F8F80C220821534800F0F3F80C227A
:100BA0000921514800F0EEF80C220A214E4800F0CD
:100BB000E9F80C220B214C4800F0E4F80C22114615
:100BC000494800F0DFF80C220D21474800F0DAF820
:100BD0000C220E21444800F0D5F80C220F21424887
:100BE00000F0D0F80C220021404800F0CBF80C2295
:100BF00001213E4800F0C6F80C2202213B4800F0DB
:100C0000C1F80C220321394800F0BCF80C22042161
:100C1000364800F0B7F80C220521344800F0B2F84D
:100C20000C221146314800F0ADF80C220D212F485E
:100C300000F0A8F80C220E212C4800F0A3F80C229A
:100C40000F212A4800F09EF80C220021284800F0CD
:100C500099F80C220121264800F094F80C22022178
:100C6000234800F08FF80C220321214800F08AF875
:100C70000C2204211E4800F085F80C2205211C4896
:100C800000F080F80C220A21194800F07BF80020BF
:100C90000190029008200390002004900590069097
:100CA000079004200890002009900A9010200B90D3
:100CB00000200C900E900D900F9010904FF48050EB
:100CC0001190002012901390149001A81590169086
:100CD00008A8FFF74BFE01210420FFF72DFE19B0F5
:100CE00000BD0000000C0240001002400014024051
:100CF00000180240F0B50A4600210023002400BF7E
:100D00003DE0012505FA01F3156805EA03049C425C
:100D100034D105684F000326BE40B5430560157900
:100D20004E00B5400668354305601579012D02D0A7
:100D30001579022D16D185684F000326BE40B543B4
:100D4000856055794E00B5408668354385604568B5
:100D500001268E40B5434560456896798E40B6B20F
:100D600035434560C5684F000326BE40B543C560A6
:100D7000D5794E00B540C6683543C560491C102979
:100D8000BFD3F0BDF0B5002300244D07ED0E02FAED
:100D900005F3CE1000F1200555F826504E07F70E4A
:100DA0000F26BE40B543CF1000F1200646F827506D
:100DB000CE1000F1200555F8265045EA0304CE1068
:100DC00000F1200545F82640F0BD418370470183BE
:100DD0007047000070B502460C46FF25FF2309E06E
:100DE00012F8010B80EA03010648405C80EA050323
:100DF0000548455C201EA4F10106B4B2F0D143EAD7
:100E0000052070BDDA1B0008DA1C000838B5FFF7B2
:100E100055FC4FF6FF74462000F0A6FB30215148E8
:100E200000F0AAFD462000F09FFB15214E4800F07F
:100E3000A3FD462000F098FB25214C4800F09CFDC6
:100E4000462000F091FB1E21494800F095FD462008
:100E500000F08AFB2521474800F08EFD462000F077
:100E600083FB30213F4800F087FD78E0424800785E
:100E7000002874D0042241A14148FFF7CDFA58B9A7
:100E80000521404800F078FD3F4800900422694663
:100E90003E4800F0BBF95AE006223DA13848FFF772
:100EA000BBFA002844D10521364800F065FDFFF764
:100EB00005FC00203049087000BF2F480078012849
:100EC000FBD1354935A0FFF7FFF905212D4800F08A
:100ED00053FD31480088801E81B22948FFF77AFF10
:100EE0000446214633A0FFF7EFF92B480068401E67
:100EF0002349095C28480068801E214A105C41EAA9
:100F00000020A0420BD124480068821E1C492C48B6
:100F100000F07CF919212B4800F02EFD03E016218A
:100F2000294800F029FD214628A0FFF7CDF90EE061
:100F3000072229A11248FFF76FFA20B905211148AD
:100F400000F01AFD0CE01A21254800F015FDFFF70E
:100F5000B5FB002008490870032000F0C1FB85E7BD
:100F600000BF38BDEA0000206D0000208200002094
:100F7000A7000020C50000200C00002041434B00CA
:100F8000000000681A010020CDAB341200400008B8
:100F90005354415254000000040000207265636500
:100FA000697665202564204279746573206D7367C6
:100FB0000D0A00004341434C203D2025780D0A00D6
:100FC00000000108240000203D000020435243207F
:100FD0003D2025780D0A000043414E43454C00005A
:100FE0005300002070B5002100230F22C4781CB3E9
:100FF000174C246804F4E064C4F5E064C4F30721EA
:10100000C1F10404E3B20A4144789C40E1B284781F
:10101000144021430C07210E0E4C057861550478CD
:1010200004F01F050124AC4005786D11AD0005F1F9
:10103000E025C5F8004109E0047804F01F0501240B
:10104000AC40054D0678761145F8264070BD00008D
:101050000CED00E000E400E080E100E00249014323
:10106000024A1160704700000000FA050CED00E034
:1010700029B1064A12680243044B1A6004E0034A8D
:1010800012688243014B1A607047000030380240FA
:1010900029B1064A12680243044B1A6004E0034A6D
:1010A00012688243014B1A607047000038380240D2
:1010B00029B1064A12680243044B1A6004E0034A4D
:1010C00012688243014B1A607047000040380240AA
:1010D00029B1064A12680243044B1A6004E0034A2D
:1010E00012688243014B1A60704700004438024086
:1010F000F0B5002100220024022500260223324FF1
:101100003F6807F00C0121B1042905D0082937D127
:1011100005E02E4F076036E02D4F076033E02A4F81
:101120003F1F3F68C7F38056274F3F1F3F6807F0B8
:101130003F036EB1264FB7FBF3F7DFF88CC0ACF17D
:10114000040CDCF800C0CCF3881C07FB0CF40CE0AA
:101150001E4FB7FBF3F7DFF870C0ACF1040CDCF8FE
:1011600000C0CCF3881C07FB0CF4174F3F1F3F68EF
:10117000C7F301477F1C7D00B4FBF5F7076002E071
:10118000124F076000BF00BF0F4F3F6807F0F0012C
:101190000909104F7A5C0768D74047600A4F3F68DB
:1011A00007F4E051890A0B4F7A5C4768D7408760A3
:1011B000054F3F6807F46041490B064F7A5C47686A
:1011C000D740C760F0BD0000083802400024F4009A
:1011D00040787D010D00002010B5044620680749C5
:1011E0000840B0F1005F08D16068054908602068D8
:1011F000FFF747F802480068804710BD0000FE2F47
:101200002000002001460868704700002DE9F047E3
:1012100004460E4617464FF009080025A94604F07B
:10122000030008B1BDE8F087FFF762FB0020FFF77D
:10123000ADFA254604EB07091748854215D2174831
:1012400085420AD102212020FFF7B2FA804602210E
:101250002820FFF7ADFA804607E01148854204D107
:1012600002210820FFF7A4FA8046B8F1090F0CD13B
:1012700008E020463168FFF713FB092800D003E09F
:10128000241D361D4C45F4D300BF0120FFF77EFA24
:10129000FFF7FCFA00BFC5E70000FF1F00000108D0
:1012A000004000080CB50020019000903448006810
:1012B00040F480303249086000BF3148006800F4D3
:1012C000003000900198401C0190009818B90198D6
:1012D000B0F5A04FF1D12A48006800F4003010B1F9
:1012E0000120009001E0002000900098012846D1E4
:1012F00023484030006840F0805021494031086068
:101300002048006840F440401E4908601C480830EE
:1013100000681B49083108600846006840F4004036
:1013200008600846006840F4A05008601648091F8D
:101330000860081F006840F08070091F086000BF47
:101340000F48006800F000700028F9D040F20570E6
:101350000E4908600A480830006820F00300084978
:10136000083108600846006840F00200086000BFCD
:1013700003480830006800F00C000828F8D10CBDC4
:10138000003802400070004019544004003C024004
:1013900002480068401C01490860704708000020AE
:1013A00010B51548006840F47000134908601348F0
:1013B000006840F001001149086000200F49083121
:1013C00008600E4800680E4908400C4908600D4846
:1013D000091D0860081F006820F48020091F0860AC
:1013E000002006490C310860FFF75CFF4FF00060F9
:1013F00001498039086010BD88ED00E000380240E6
:10140000FFFFF6FE103000247FB505460C46012193
:101410000220FFF74DFE0295ADF804400020ADF824
:101420000600ADF80C0001A90C4800F05BF80121A2
:101430000A4800F02DF801221146084800F048F84B
:101440001D208DF8000001208DF801008DF80200AC
:101450008DF803006846FFF7C5FD7FBD000400401E
:1014600010B50121084800F022F8012806D100211A
:10147000054800F010F801200449087001210248D5
:1014800000F006F810BD0000000400400C00002031
:10149000CA430282704721B1028842F001020280F1
:1014A00004E002884FF6FE731A400280704730B5A0
:1014B0000246002000230024158A05EA01039589CD
:1014C00005EA010413B10CB1012000E0002030BD99
:1014D0001AB183890B43838102E083898B43838123
:1014E0007047000000220288184B98420ED0184B1B
:1014F00098420BD0B0F1804F08D0164B984205D0DF
:10150000154B984202D0154B984204D14FF68F7379
:101510001A404B881A43124B984207D0114B9842FD
:1015200004D04FF6FF431A400B891A4302804B68E0
:10153000C3620B880385054B984202D0044B984246
:1015400001D18B7A0386012383827047000001401A
:10155000000401400004004000080040000C00406E
:101560000010004000140040044A116800BF034A04
:101570001268521A8242FAD3704700000800002015
:1015800010B588B0044601210C20FFF771FD012140
:101590000805FFF78DFD082202213648FFF7F2FB10
:1015A00008220C213448FFF7EDFB042006900220AE
:1015B0008DF81C008DF81D0000208DF81E00012004
:1015C0008DF81F0006A92B48FFF794FB4FF48050BD
:1015D000069002208DF81C008DF81D0000208DF86B
:1015E0001E0001208DF81F0006A92348FFF782FB8B
:1015F0000820069001208DF81C0002208DF81D00A7
:1016000000208DF81E0001208DF81F0006A9194842
:10161000FFF770FB032000F063F802940020ADF8A0
:101620000C00ADF80E00ADF81000ADF814000C2061
:10163000ADF8120002A9114800F030F901210F485D
:1016400000F0D1F8012240F225510C4800F001F9D8
:1016500035208DF8040005208DF8050000208DF858
:10166000060001208DF8070001A8FFF7BBFC08B0B9
:1016700010BD0000000C0240000802400050004075
:1016800010B540F22551124800F0B9F8D0B1104819
:101690008088C1B20F4802680068401C0D4B18607A
:1016A0000D48815400200D49086001210B48243861
:1016B000FFF7F1FE07480068B0F5483F02D100206F
:1016C0000449086040F22551014800F07DF810BD42
:1016D0000050004004000020000000682404004086
:1016E00010B50446022C04D108210548FFF76FFB12
:1016F00005E0032C03D108210148FFF766FB10BD6C
:10170000000C024010B588B0044601210846FFF7DE
:10171000AFFC01211020FFF7DBFC07220921234841
:10172000FFF730FB07220A212048FFF72BFB4FF47D
:10173000C060069002208DF81C008DF81D0000206E
:101740008DF81E0001208DF81F0006A91748FFF72D
:10175000D1FA02940020ADF80C00ADF80E00ADF8FF
:101760001000ADF814000C20ADF8120002A91048CA
:1017700000F094F801210E4800F035F8012240F203
:1017800025510B4800F065F825208DF80400032052
:101790008DF8050000208DF8060001208DF8070067
:1017A00001A8FFF71FFC08B010BD000000000240B8
:1017B0000010014010B540F22551024800F004F835
:1017C00010BD00000010014010B50022002340F6BB
:1017D0006A14A14200D100BF0A1201249440A3B2AE
:1017E000DC43048010BD21B1828942F40052828121
:1017F00004E082894DF6FF731A408281704770B50C
:101800000246002400230025002040F66A16B1425B
:1018100000D100BFC1F3421501F01F03012606FAF3
:1018200003F3012D02D19689334006E0022D02D147
:10183000168A334001E0968A33400C12012606FADC
:1018400004F41688344013B10CB1012000E00020EC
:1018500070BDF0B50346002400260025002040F6A8
:101860006A17B94200D100BF1846C1F3421401F013
:101870001F06012707FA06F5012C01D10C3004E000
:10188000022C01D1103000E014301AB107682F4348
:10189000076002E00768AF430760F0BD2DE9FF472E
:1018A00005460E460024A14600BFA046B08900B1FF
:1018B00000BF2C8A24F44054F08804432C82AC8965
:1018C00041F20C608443B088318908437189084330
:1018D0000443AC81AC8A24F44074B0890443AC82E4
:1018E0006846FFF705FC2048854202D01F48854224
:1018F00002D1DDF80C9001E0DDF80890A88900F431
:10190000004040B109EBC90000EB09103168490003
:10191000B0FBF1F707E009EBC90000EB09103168F3
:101920008900B0FBF1F76420B7FBF0F00401200957
:10193000642101FB1078A88900F4004040B13220F6
:1019400000EBC800B0FBF1F000F00700044308E032
:10195000322000EB08106421B0FBF1F000F00F0022
:1019600004432C81BDE8FF870010014000140140B2
:10197000C1F308028280704770B505460E4602200A
:10198000FFF7AEFE0120FFF7EFFD00240CE0295D1C
:101990000A48FFF7EDFF00BF0848008800F040004C
:1019A0000028F9D0601CC4B2B442F0DB0120FFF77C
:1019B000DBFD0320FFF794FE70BD000000500040E7
:1019C00000BF704700BF054A128802F04002002A9B
:1019D000F9D0C2B2014B9A8070470000001001405C
:1019E00008B54FF44070FFF739FBFEF775FE4FF472
:1019F000E130FFF787FE4FF4E130FFF7C1FD4FF410
:101A000000610846FFF700FDFFF724F82DA0FEF760
:101A10005BFC4FF448313448FEF749FDFEF78CFE7D
:101A20003248FFF7EFFB00900098B0F1FF3F2BD05A
:101A30002F49084420B12F490844002833D109E038
:101A40002DA0FEF741FC1420FFF78EFD3548FFF76F
:101A5000C3FB2CE034A0FEF737FC3E4800904FF467
:101A6000003230480099FFF7D1FB0A20FFF77CFDD8
:101A70001F4840420090042269461C48FFF7C6FBFD
:101A80002848FFF7A9FB12E033A0FEF71DFC184819
:101A900040420090042269461448FFF7B7FB2148F2
:101AA000FFF79AFB03E037A0FEF70EFC00BF00BF74
:101AB00006E040A0FEF708FC41F28830FFF754FD35
:101AC000F7E700000D0A2A2A2A2A2A2A2A2A2A2A7D
:101AD000426F6F744C6F616465722A2A2A2A2A2A1F
:101AE0002A2A2A2A0D0A0000000000680040000887
:101AF0003354CBED1201CDCC0D0A2A2A2A2A2A2AE8
:101B00002A2A2A2A52756E696E67204669726D7795
:101B1000617265202A2A2A2A2A2A2A2A2A2A0D0AB2
:101B200000000000000001080D0A2A2A2A2A2A2A99
:101B30002A2A2A2A4C6F6164696E67204669726D91
:101B400077617265202A2A2A2A2A2A2A2A2A2A0D15
:101B50000A000000000004080D0A2A2A2A2A2A2A5C
:101B60002A2A2A2A44656661756C74204669726D5A
:101B700077617265202A2A2A2A2A2A2A2A2A2A0DE5
:101B80000A0000000D0A2A2A2A2A2A2A2A2A2A2A90
:101B9000446F6E5E7420486176696E672046697294
:101BA0006D77617265202A2A2A2A2A2A2A2A2A2A55
:101BB0000D0A00000D0A2A2A2A2A2A2A2A2A49441A
:101BC0004C452A2A2A2A2A2A2A2A0D0A000000001D
:101BD0004FF04070E1EE100A704700C1814001C033
:101BE000804101C0804100C1814001C0804100C1ED
:101BF000814000C1814001C0804101C0804100C1DD
:101C0000814000C1814001C0804100C1814001C0CC
:101C1000804101C0804100C1814001C0804100C1BC
:101C2000814000C1814001C0804100C1814001C0AC
:101C3000804101C0804100C1814000C1814001C09C
:101C4000804101C0804100C1814001C0804100C18C
:101C5000814000C1814001C0804101C0804100C17C
:101C6000814000C1814001C0804100C1814001C06C
:101C7000804101C0804100C1814000C1814001C05C
:101C8000804101C0804100C1814001C0804100C14C
:101C9000814000C1814001C0804100C1814001C03C
:101CA000804101C0804100C1814001C0804100C12C
:101CB000814000C1814001C0804101C0804100C11C
:101CC000814000C1814001C0804100C1814001C00C
:101CD000804101C0804100C1814000C0C101C303F7
:101CE00002C2C60607C705C5C404CC0C0DCD0FCF74
:101CF000CE0E0ACACB0BC90908C8D81819D91BDBE4
:101D0000DA1A1EDEDF1FDD1D1CDC14D4D515D71733
:101D100016D6D21213D311D1D010F03031F133F3E3
:101D2000F23236F6F737F53534F43CFCFD3DFF3F33
:101D30003EFEFA3A3BFB39F9F83828E8E929EB2B63
:101D40002AEAEE2E2FEF2DEDEC2CE42425E527E7F3
:101D5000E62622E2E323E12120E0A06061A163A363
:101D6000A26266A6A767A56564A46CACAD6DAF6FF3
:101D70006EAEAA6A6BAB69A9A86878B8B979BB7B63
:101D80007ABABE7E7FBF7DBDBC7CB47475B577B7B3
:101D9000B67672B2B373B17170B0509091519353E3
:101DA000529296565797559594549C5C5D9D5F9FB3
:101DB0009E5E5A9A9B5B99595898884849894B8BE3
:101DC0008A4A4E8E8F4F8D4D4C8C44848545874773
:101DD00046868242438341818040303132333435FC
:101DE0003637383941424344454640305800303157
:101DF0003233343536373839616263646566403072
:101E000078000000241E00080000002034010000BB
:101E1000C4010008F01E0008340100206404000022
:101E20002002000801112D010203040475060708B1
:101E300009E81946697265576172652043686563F0
:101E40006B20537563636573730D0A191D466169D1
:101E50006C161818496E70757420436F6D6D616E45
:101E60006420496E636F72726563741A1D434D443A
:101E70000901180C4465736372697074696F6E159B
:101E80001E53544152541668135374617274205592
:101E900070205472616E736D6974205F19251D4145
:101EA000434B3A24A80C436F6E6669726D205468E8
:101EB000651E2F43414E43454C203E616E63656C69
:101EC0001F180F5570646174652050726F677261DE
:101ED0006D250C280D0A2A0119301B4F4B05580C93
:101EE000456E746572204C6F63616C521915000069
:040000050800018965
:00000001FF
